:100000000C94F4000C9415010C9415010C9415013A
:100010000C9415010C9415010C9415010C94150108
:100020000C9415010C9415010C9415010C941501F8
:100030000C9415010C9415010C9415010C941501E8
:100040000C9415010C9415010C9415010C941501D8
:100050000C9415010C9415010C9415010C941501C8
:100060000C9415010C9415010C9415010C941501B8
:100070000C9415010C9415010C9415010C941501A8
:100080000C9415010C9415010C9415010C94150198
:100090000C9415010C9415010C9415010C94150188
:1000A0000C9415010C9415010C9415010C94150178
:1000B0000C9415010C9415010C9415010C94692DE8
:1000C0000C9415010C9415010C9415010C94150158
:1000D0000C9415010C94E5420C9415010C94150137
:1000E0000C9415010C9415010C9415010C94150138
:1000F0000C9415010C9415010C9415010C94150128
:100100000C9415010C9415010C9415010C94150117
:100110000C9415010C9415010C9415010C94150107
:100120000C9415010C9415010C9415010C941501F7
:100130000C9415010C94E9360C9415010C941501DE
:100140000C9415010C9415010C9415010C948A3033
:100150000C9415010C9415010C9415010C941501C7
:100160000C9415010C9415010C9415010C941501B7
:100170000C9415010C9415010C9415010C941501A7
:100180000C9415010C9415010C9415010C94150197
:100190000C9415010C9415010C9415010C94150187
:1001A0000C9462360C9415010C9415010C941501F5
:1001B0000C94D52E0C9415010C9415010C9415017A
:1001C0000C9415010C9415010C9415010C94150157
:1001D0000C9415010C9415010C9415010C94150147
:1001E0000C9415010C94150111241FBECFEFDFE50F
:1001F000DEBFCDBF00E00CBF17E2A0E0B0E2E0EA56
:10020000FFE800E00BBF02C007900D92A436B107D3
:10021000D9F71BE5A4E6B7E201C01D92A330B107F0
:10022000E1F70E9410410C94CE470C9400000F930C
:10023000DF93CF930F92CDB7DEB72FB72983F89412
:100240001BBEFC0108ED04BF608389818FBF0F9046
:10025000CF91DF910F91089520911D01922F80E0A1
:1002600080937F279093802780917F27909180278C
:1002700020911C01820F911D80937F2790938027EE
:1002800080917F279091802789579D4480937F2775
:100290009093802720917F273091802780917D2720
:1002A00090917E2740E02817390709F041E0842F1C
:1002B00008950E942C01882331F120911D01922F75
:1002C00080E080937F279093802780917F27909173
:1002D000802720911C01820F911D80937F2790938E
:1002E000802780917F279091802789579D44809314
:1002F0007F279093802780917F27909180278093FC
:100300007D2790937E270895AB01BC01E0E0F1E0EA
:1003100080910001806880930001809112018560C6
:10032000828B8BE4838B84E690E0848B958B168A9A
:1003300080EA808F28E0218F128E89E79DE4848FE8
:10034000958F168E80911001846A808BE0E4F6E030
:10035000218384E0828391E0928382E0818386839B
:10036000E0EAF8E083E08583403825E2520720E0A8
:10037000620720E0720711F48FE509C0403022ECDB
:10038000520721E0620720E0720719F487E08683B4
:1003900018C0403024E8520723E0620720E07207CB
:1003A000B1F3403088E0580787E0680780E07807BD
:1003B00011F4968306C0405050416E40704011F4D5
:1003C00016821782E0EAF8E08091A40880618483B5
:1003D0008091A408886084830E945901089588232D
:1003E00021F00E942C018823E1F3E0917D27F09118
:1003F0007E27E758F24BE08180917D2790917E2700
:10040000019680937D2790937E2780917D27909100
:100410007E278436910520F010927D2710927E274A
:100420008E2F0895482F8091A10885FFFCCF2EC004
:100430008091812790918227A0918327B091842772
:100440000196A11DB11D8093812790938227A093CF
:100450008327B09384278091812790918227A09150
:100460008327B091842781519742A040B04050F03B
:10047000109281271092822710928327109284274E
:1004800080E00895C9010197F1F702C026E63EE039
:100490008091480680FDCCCF4093A00881E008956C
:1004A000E82FF0E081E090E00E2E02C0880F991F47
:1004B0000A94E2F7A0EAB6E011968C93ED58F84C56
:1004C00010820895E3E7F7E3E80FF11D60830895D4
:1004D00021E030E002C0220F331F8A95E2F7E0EA04
:1004E000F6E02583089521E030E002C0220F331F9B
:1004F0008A95E2F7E0EAF6E02683089521E030E00D
:1005000002C0220F331F8A95E2F7E0EAF6E0278364
:10051000089588E08093400880EC80938001E0E0BB
:10052000F8E08FEF9FEF86A397A38081807F8460A0
:10053000808308950F93DF93CF930F92CDB7DEB7EB
:10054000AB01BC01F89482E08093F0008FB78983FF
:10055000F8941BBE21E080EF90E0FC0108ED04BFA1
:10056000208389818FBF8091F00084608093F000A8
:100570008091F00088608093F000809120048E7F4D
:1005800080932004E0E2F4E08091210480FDFACF22
:100590008EEF9FEFAFEFBFEF80879187A287B38782
:1005A000148615861686178644835583668377835B
:1005B00080E090E90197F1F781E080932004809139
:1005C000210480FDFCCF80912204837F8460E0E2DF
:1005D000F4E0828378940F90CF91DF910F9108958A
:1005E0008091F10087FD12C08091F10080FD0EC066
:1005F0008091F10081FD0AC082E08093F00080913B
:10060000F1008695869580958170089580E0089523
:10061000809121048061E0E2F4E0818380912104F3
:1006200084FDFCCF209124043091250440912604C0
:1006300050912704B901CA010895F89420916008E7
:1006400030916108609120087091210880916008C4
:10065000909161082817390741F020916008309186
:1006600061086091200870912108789440E050E082
:10067000A90133272227CB01A0E0B0E0280F391FC2
:100680004A1F5B1FB901CA0108958F929F92AF92D2
:10069000BF92CF92DF92EF92FF920F931F93CF936F
:1006A000DF937B018C01EA012CE330E040E050E075
:1006B0000E9475466983C801B7012CE330E040E031
:1006C00050E00E947546122F032FF42EE52E622F64
:1006D000732F842F952F2CE330E040E050E00E94F0
:1006E00075466A83612F702F8F2D9E2D2CE330E08D
:1006F00040E050E00E947546122F032FF42EE52EA5
:10070000622F732F842F952F28E130E040E050E0D6
:100710000E9475466B83612F702F8F2D9E2D28E1CF
:1007200030E040E050E00E94754679018A01C8013E
:10073000B7016C5F7F4F8F4F9F4F27E030E040E065
:1007400050E00E9475466F5F6C8320E0AA24BB24B2
:10075000650101C02F5F822E9924F401EE54F84FF9
:10076000CF0183709070892B99F4CF0164E670E01B
:100770000E946246892B39F4CF0160E971E00E9442
:100780006246892B29F48EE691E0A0E0B0E004C037
:100790008DE691E0A0E0B0E0A80EB91ECA1EDB1EF7
:1007A000C501A0E0B0E0E816F9060A071B0790F6BD
:1007B0002F83F401EE54F84F93E0892E912C8E2272
:1007C0009F228114910499F4CF0164E670E00E94A5
:1007D0006246892B39F4CF0160E971E00E946246DC
:1007E000892B29F48EE691E0A0E0B0E004C08DE60C
:1007F00091E0A0E0B0E0A81AB90ACA0ADB0A9801A1
:1008000087010A191B092C093D09CF0164E670E034
:100810000E9462467C01CF0160E971E00E9462465D
:10082000AC01E8E5F7E260E0613051F48114910435
:1008300049F4E114F10441F44115510529F002C0D5
:10084000808103C08CE101C08DE190E0A0E0B0E0C8
:10085000081719072A073B0740F0081B190B2A0B3A
:100860003B0B6F5F31966C30F9F66F5F6E83802FB4
:100870008F5F8D83CE01DF91CF911F910F91FF90FC
:10088000EF90DF90CF90BF90AF909F908F900895A2
:1008900082E38093C8278FEFE0ECF9E083838091B7
:1008A000C20987FFFCCF8091C309E0ECF9E02FEF8C
:1008B00023838091C20987FFFCCF9091C3099F3F9A
:1008C00021F08091C827882399F7892F08951F93D5
:1008D000CF93DF93C0E6D6E010E11E830E94480468
:1008E0008F3F11F481E00CC01D838FEFE0ECF9E045
:1008F00083838091C20987FFFCCF8091C30980E088
:10090000DF91CF911F910895FC0184E18093C72767
:10091000A0ECB9E09FEF13969C9313978091C209C6
:1009200087FFFCCF8091C3098F3F29F48091C727AF
:10093000882389F749C08E3F09F046C0A0ECB9E092
:100940009FEF13969C9313978091C20987FFFCCF6A
:100950008091C309808313969C9313978091C20959
:1009600087FFFCCF8091C309818313969C931397D3
:100970008091C20987FFFCCF8091C30982831396BF
:100980009C9313978091C20987FFFCCF8091C30984
:1009900083836450704011F03496D3CF8FEFE0EC36
:1009A000F9E083838091C20987FFFCCF8091C3095E
:1009B0008FEFE0ECF9E083838091C20987FFFCCFE1
:1009C0008091C30981E0089580E008951F93CF933B
:1009D000DF93EC01162F0E9448048F3F11F090E046
:1009E0003FC0E0ECF9E013838091C20987FFFCCFA0
:1009F0001D3F11F491E034C090E0E0ECF9E0888113
:100A000083838091C20987FFFCCF89818383809192
:100A1000C20987FFFCCF915011F02296F0CF8FEFE3
:100A2000E0ECF9E083838091C20987FFFCCF8FEF70
:100A3000E0ECF9E083838091C20987FFFCCF8FEF60
:100A4000E0ECF9E083838091C20987FFFCCF8091BD
:100A5000C30990E08F71853009F091E081E098271B
:100A6000892FDF91CF911F910895DF92EF92FF922E
:100A70000F931F93D82E7A018B0187FF0CC087E755
:100A800040E050E060E070E00E943505823008F000
:100A900072C08FE7D82280E1E0E6F6E085838FEF31
:100AA000E0ECF9E083838091C20987FFFCCF80915D
:100AB000C3090E946704882311F48FEF5CC0E0EC47
:100AC000F9E0D3828091C20987FFFCCF812F99275B
:100AD000AA27BB27E0ECF9E083838091C20987FF56
:100AE000FCCFC801AA27BB27E0ECF9E08383809103
:100AF000C20987FFFCCFBB27A12F902F8F2DE0ECE1
:100B0000F9E083838091C20987FFFCCFE0ECF9E034
:100B1000E3828091C20987FFFCCF80E4D81611F4EC
:100B200085E906C088E4D81611F487E801C081E0A1
:100B3000E0ECF9E083838091C20987FFFCCF8CE46D
:100B4000D81651F48FEFE0ECF9E083838091C2096D
:100B500087FFFCCF8091C3099AE0E0ECF9E02FEF2A
:100B600023838091C20987FFFCCF8091C30987FF4F
:100B700002C09150A9F71F910F91FF90EF90DF9065
:100B80000895EF92FF920F931F93DF93CF9300D0BE
:100B90000F92CDB7DEB78091572781FDCCC0E0E63C
:100BA000F6E080EB818388E3868B14828CE291E00F
:100BB00020E731E0F9013197F1F70197D9F783E5A3
:100BC0008093C0099AE0E0ECF9E02FEF2383809155
:100BD000C20987FFFCCF8091C3099150B9F780E427
:100BE00040E050E060E070E00E943505813009F09F
:100BF00087C084E68093C72788E44AEA51E060E032
:100C000070E00E943505813009F053C07E010894E0
:100C1000E11CF11C8701E0ECF9E09FEF9E012B5FE6
:100C20003F4F93838091C20987FFFCCF8091C30916
:100C3000D8018D938D01A217B30799F78B8181306D
:100C400009F05EC08C818A3A09F05AC08091C727AA
:100C5000882349F089EE40E050E060E070E40E94B3
:100C60003505882399F78091C727882309F448C060
:100C70008AE740E050E060E070E00E94350588239C
:100C800009F03EC0E0ECF9E09FEF93838091C20948
:100C900087FFFCCF8091C309D7018D937D01A017F9
:100CA000B10799F7898186FD02C014E02AC01CE0D3
:100CB00028C089EE40E050E060E070E00E94350519
:100CC000823018F001E411E002C009EE12E08091D8
:100CD000C727882349F0802F40E050E060E070E0B3
:100CE0000E943505882399F78091C727882341F012
:100CF00080E540E052E060E070E00E94350581113F
:100D000010E01093C92780E1E0E6F6E085838FEFDD
:100D1000E0ECF9E083838091C20987FFFCCF8091EA
:100D2000C309112341F0809157278E7F8093572765
:100D300080ED8093C009809157272496CDBFDEBFF8
:100D4000CF91DF911F910F91FF90EF90089588232D
:100D500011F081E008958091572708950F93CF9364
:100D6000DF93EB01882309F053C0002309F450C03E
:100D70008091572780FF02C003E04BC08091C927B4
:100D800083FD07C069E0220F331F441F551F6A957A
:100D9000D1F7013089F481E5BA01A9010E94350536
:100DA000882321F5CE0160E072E00E94840400E017
:100DB0008823E1F401E01AC082E5BA01A9010E948A
:100DC0003505882399F4CE0160E072E00E94840426
:100DD000882329F0015019F0C050DE4FF4CF8CE485
:100DE00040E050E060E070E00E94350580E1E0E620
:100DF000F6E085838FEFE0ECF9E083838091C20910
:100E000087FFFCCF8091C309002319F001E001C0E6
:100E100004E0802FDF91CF910F910895CF92DF9260
:100E2000EF92FF920F93CF93DF93EB0169017A0169
:100E3000882309F061C0002309F45EC08091572720
:100E400080FF02C003E059C08091572782FF02C093
:100E500002E053C08091C92790E083FD07C079E08C
:100E6000CC0CDD1CEE1CFF1C7A95D1F7013069F427
:100E700088E5B701A6010E943505882359F5CE0102
:100E80006EEF0E94E60400E022C086709070892B0D
:100E900039F0402F50E060E070E087ED0E943505AA
:100EA00089E5B701A6010E943505882399F4CE0192
:100EB0006CEF0E94E604882329F0015019F0C0501D
:100EC000DE4FF5CF80E090E06DEF0E94E6048823CE
:100ED00009F401E080E1E0E6F6E085838FEFE0ECE5
:100EE000F9E083838091C20987FFFCCF8091C30919
:100EF000002319F001E001C004E0802FDF91CF91C1
:100F00000F91FF90EF90DF90CF900895FF920F9395
:100F10001F93DF93CF93CDB7DEB76097CDBFDEBF12
:100F20008A01882309F0B8C1643001F5FA01808193
:100F3000813039F0813008F4B1C1823009F0ACC1A0
:100F400011C0E0E6F6E080EB818388E3868B1482B3
:100F50008CE291E020E731E0F9013197F1F7019758
:100F6000D9F79CC181E0FA01818398C1809157270C
:100F700080FF02C093E093C16A3009F42FC16B3047
:100F800050F4613051F16130A0F0623009F486C054
:100F9000633069F489C06C3009F427C16C3008F4FF
:100FA00022C16D3009F42EC16E3009F44AC194E0BB
:100FB00064C10E946704882309F45EC180E1E0E611
:100FC000F6E085838FEFE0ECF9E083838091C2093E
:100FD00087FFFCCF8091C309FFC089E440E050E067
:100FE00060E070E00E943505882309F045C1CE011C
:100FF000019660E170E00E948404882309F43CC1FA
:10100000898182958695869583707A854985813018
:1010100089F4872F90E00196342F20E0820F931FF0
:10102000A0E0B0E02AE0880F991FAA1FBB1F2A95F5
:10103000D1F7CDC04295469546954370288530E05E
:10104000220F331F220F331F240F311D2F5F3F4FFD
:101050008F8190E083709070982F8827990F990F57
:10106000280F391F40E050E08E818F706B85661F1E
:101070006627661F860F8E5F7370770F870F90E06D
:10108000099704C0220F331F441F551F8A95D2F7BA
:10109000F80120833183428353839EC080E092E035
:1010A000FA018083918398C08091C927F82E82FF2E
:1010B00039C08DEC40E050E060E070E00E94350502
:1010C000882309F0D9C08FEFE0ECF9E083838091A9
:1010D000C20987FFFCCF8091C309CE01019660E170
:1010E00070E00E948404882309F4C6C090E3E0EC19
:1010F000F9E02FEF23838091C20987FFFCCF809115
:10110000C3099150B9F72B8522952F7080E190E0AB
:10111000A0E0B0E004C0880F991FAA1FBB1F2A954A
:10112000D2F755C089E440E050E060E070E00E94F2
:101130003505882309F0A0C0CE01019660E170E07A
:101140000E948404882309F497C04B858C85F1FEA6
:101150001BC0881F8827881F90E00196242F30E04D
:101160002F733070220F331F820F931F2E8522950D
:1011700026952695237030E02150304002C0880F1C
:10118000991F2A95E2F721C0282F30E02370307094
:10119000F3E0220F331FFA95E1F782958695877069
:1011A000280F311D2F5F3F4F842F90E08C77907078
:1011B00095958795959587950196AC01249FC001DB
:1011C000259F900D349F900D1124A0E0B0E0F80110
:1011D00080839183A283B38390E04FC08091C9271D
:1011E000FA018083F9CF89E401C08AE440E050E04D
:1011F00060E070E00E9435058823F1F5C80160E1E8
:1012000070E035C08AE740E050E060E070E00E94A6
:101210003505882389F5F801A0ECB9E09FEF980126
:101220002D5F3F4F13969C9313978091C20987FFC0
:10123000FCCF8091C3098083E217F30769F23196EE
:10124000F1CF8DEC40E050E060E070E00E943505A9
:10125000882391F48FEFE0ECF9E083838091C20959
:1012600087FFFCCF8091C309C80160E470E00E9451
:10127000840490E0882309F491E080E1E0E6F6E060
:1012800085838FEFE0ECF9E083838091C20987FFCB
:10129000FCCF8091C30903C094E001C090E0892F86
:1012A0006096CDBFDEBFCF91DF911F910F91FF9070
:1012B00008958091C727882319F081508093C7270C
:1012C0008091C827882319F081508093C827809186
:1012D0005727897F809357270895EF92FF920F93A6
:1012E0001F93DF93CF93CDB7DEB72897CDBFDEBF77
:1012F0006091852770918627809187279091882714
:101300006054784380409040AE014F5F5F4F0E9431
:101310004503888590E00A977C010027F7FC00953B
:10132000102FA9E1EE0CFF1C001F111FAA95D1F789
:101330002E8130E040E050E0A901332722278F8141
:1013400090E0A0E0B0E0E5E1880F991FAA1FBB1F65
:10135000EA95D1F7282B392B4A2B5B2B8C8190E017
:10136000A0E0B0E07BE0880F991FAA1FBB1F7A9511
:10137000D1F7282B392B4A2B5B2B8B8190E0A0E0F7
:10138000B0E065E0880F991FAA1FBB1F6A95D1F7CF
:10139000282B392B4A2B5B2B8A81869590E0A0E085
:1013A000B0E0282B392B4A2B5B2B2E293F29402BD1
:1013B000512BB901CA012896CDBFDEBFCF91DF9175
:1013C0001F910F91FF90EF9008956F927F928F92EF
:1013D0009F92AF92BF92CF92DF92EF92FF920F93C4
:1013E0001F93CF93DF93EC014A015B01CAA4DBA4F6
:1013F000ECA4FDA4C416D506E606F70609F44EC013
:101400008C818823A1F1BEE26B2E712C6C0E7D1EA7
:101410008981B301A701960101E00E940E0788238C
:10142000D9F51C828E899F89A88DB98D2E8D3F8D0F
:1014300048A159A1820F931FA41FB51FC816D90632
:10144000EA06FB06A0F41B8110C08E899F89A88D37
:10145000B98DC80ED91EEA1EFB1E8981B301A701F2
:10146000960101E00E940E071150123070F78114AE
:101470009104A104B10491F0BE01625D7F4F8981A6
:10148000A501940101E00E94AE06882329F48AA6F2
:101490009BA6ACA6BDA603C081E001C080E0DF91A1
:1014A000CF911F910F91FF90EF90DF90CF90BF9061
:1014B000AF909F908F907F906F9008950F93CF93F0
:1014C000DF93EC0140E050E060E070E00E94E5094D
:1014D000882309F07EC08881833009F072C08D8135
:1014E000882309F46EC01AA61BA61CA61DA6BE0161
:1014F000625D7F4FFB0180E092E001C01192019795
:101500002FEF8F3F9207D1F7C45DDD4F85E58993BB
:101510008AEA8883CD52D24082E58EA78FA721E642
:1015200028AB91E499ABCE5EDD4F82E78993899336
:1015300099932883C551D2408E85CA5EDD4F88833A
:10154000C651D2408F85C95EDD4F8883C751D240D6
:101550008E859F85A889B9899D0144275527C85E36
:10156000DD4F288321968B2F9927AA27BB278883B5
:10157000C951D2408A85C65EDD4F8883CA51D240A8
:101580008B85C55EDD4F8883CB51D2408A859B8594
:10159000AC85BD859D0144275527C45EDD4F28835A
:1015A00021968B2F9927AA27BB278883CD51D2401C
:1015B0002A893B894C895D89898101E00E940E0757
:1015C0001D82898160E040E050E00E948607811121
:1015D00081E0DF91CF910F9108957F928F929F923A
:1015E000AF92BF92CF92DF92EF92FF920F931F9331
:1015F000CF93DF934C017A018B0142305105610595
:10160000710508F4BBC0F401828D938DA48DB58D56
:10161000481759076A077B0708F0B0C0A68CB78C3B
:10162000C0A0D1A08081823009F44DC0833009F47C
:1016300068C0813009F0A7C0EA01D695C795CE0DE4
:10164000DF1DAE01452F5527469560E070E04A0D3D
:101650005B1D6C1D7D1DC4010E94E509882309F0F6
:1016600092C0FE01F170E80DF91D76A42196AE013D
:10167000452F5527469560E070E04A0D5B1D6C1DB7
:101680007D1DC4010E94E509882309F07CC0672DF7
:1016900070E0D170C80DD91D9EA580E0682B792B14
:1016A000C70181709070892B39F094E07695679529
:1016B0009A95E1F79B0122C09B0140E050E03F700A
:1016C0004070507064C0452F562F672F77274A0D02
:1016D0005B1D6C1D7D1DC4010E94E509882309F076
:1016E00052C0F701EE0FFF1FF170E80DF91D97A52D
:1016F00080E026A530E0822B932B9C0140E050E057
:1017000046C0B7E07695679557954795BA95D1F756
:101710004A0D5B1D6C1D7D1DC4010E94E5098823D7
:1017200091F5F701EE0FFF1FEE0FFF1FF170E80DAF
:10173000F91D81A990E0A0E0B0E0582F442733279D
:10174000222780A990E0A0E0B0E0DC01992788275B
:10175000282B392B4A2B5B2B86A590E0A0E0B0E02C
:10176000282B392B4A2B5B2B97A580E0A0E0B0E01B
:10177000282B392B4A2B5B2B5F7009C021E030E00E
:1017800040E050E004C02FEF3FEF4FEF5FEFB901B3
:10179000CA01DF91CF911F910F91FF90EF90DF90E1
:1017A000CF90BF90AF909F908F907F9008952F9291
:1017B0003F924F925F926F927F928F929F92AF92E1
:1017C000BF92CF92DF92EF92FF920F931F93CF932E
:1017D000DF933C016A017B01480159014230510508
:1017E0006105710508F4BAC0F301828D938DA48D53
:1017F000B58D481759076A077B0708F0AFC0268CDC
:10180000378C40A051A08081823009F464C08330BD
:1018100009F47AC0813011F022E09CC0EA01D6952B
:10182000C795C40FD51FAE01452F5527469560E0DB
:1018300070E0420D531D641D751DC3010E94E50932
:10184000282F882309F086C0DE01B170860101705F
:1018500010700115110551F0F301EA0FFB1F86A569
:101860008F70982D9295907F982B01C0982DA60D82
:10187000B71D9E969C93219681E0F3018483AE016F
:10188000452F5527469560E070E0420D531D641DBD
:10189000751DC3010E94E509282F882309F05AC04D
:1018A000D170012B49F034E0B694A79497948794B3
:1018B0003A95D1F7482D0BC0F301EC0FFD1F46A55B
:1018C000407FBB27AB2D9A2D892D8F70482BC60DDD
:1018D000D71D4EA73FC0452F562F672F7727420DA4
:1018E000531D641D751DC3010E94E509282F88231F
:1018F00089F5F601EE0FFF1FF170E60DF71D86A6C4
:10190000892D992787A726C0B7E0769567955795C3
:101910004795BA95D1F7420D531D641D751DC3013E
:101920000E94E509282F8823A9F4F601EE0FFF1F76
:10193000EE0FFF1FF170E60DF71D86A6892D992782
:1019400087A7C501AA27BB2780AB8B2D9927AA277C
:10195000BB2781AB81E0F301848301C022E0822FA9
:10196000DF91CF911F910F91FF90EF90DF90CF907B
:10197000BF90AF909F908F907F906F905F904F90AF
:101980003F902F9008959F92AF92BF92CF92DF9297
:10199000EF92FF920F931F93CF93DF93EC017A01A5
:1019A0008B01423051056105710508F458C08A8DDC
:1019B0009B8DAC8DBD8D481759076A077B0708F4CE
:1019C00041C04DC0CE01B801A7010E94ED0A5B01E4
:1019D0006C01611571058105910509F442C081E032
:1019E000A816B104C104D104D1F12FEFA2162FEF34
:1019F000B2062FEFC2062FEFD20611F481E032C0FB
:101A0000CE01B801A70100E010E020E030E00E9424
:101A1000D70B882339F58E859F85A889B9898F3F93
:101A20002FEF92072FEFA2072FEFB20741F0019699
:101A3000A11DB11D8E879F87A88BB98B9D828601C2
:101A4000750102C0992493948A8D9B8DAC8DBD8DB8
:101A5000E816F9060A071B0708F4B4CF02C082E0B3
:101A600001C080E0DF91CF911F910F91FF90EF9027
:101A7000DF90CF90BF90AF909F9008952F923F92AC
:101A80004F925F926F927F928F929F92AF92BF928E
:101A9000CF92DF92EF92FF920F931F93DF93CF933A
:101AA00000D00F92CDB7DEB71C012A013B01DC014B
:101AB0005A968D919D910D90BC91A02D89839A830A
:101AC000AB83BC83411551056105710581F4F101BA
:101AD00082849384A484B58481149104A104B10404
:101AE00011F188169906AA06BB06E8F421C0C101C7
:101AF0000E94ED0A9B01AC016230710581059105E0
:101B000028F421E030E040E050E093C089819A81E0
:101B1000AB81BC81281739074A075B0708F489C0E5
:101B20005301420105C0A1E08A2E912CA12CB12CB9
:101B3000750164010894C11CD11CE11CF11C898150
:101B40009A81AB81BC81C816D906EA06FB0660F013
:101B500092E089169104A104B10408F461C0F2E096
:101B6000CF2ED12CE12CF12CC101B701A6010E948E
:101B7000ED0A9B01AC016115710581059105A9F084
:101B80006F3FAFEF7A07AFEF8A07AFEF9A0709F41D
:101B900050C0613071058105910509F44AC0C8142F
:101BA000D904EA04FB0431F63BC0BC2CAD2C9E2CBE
:101BB0008F2CC101A601B7010FEF1FEF2FEF3FE000
:101BC0000E94D70B882389F54114510461047104E4
:101BD00049F0C101B301A201860197010E94D70B10
:101BE000882319F5F101B286A386948685868685B9
:101BF0009785A089B1898F3FFFEF9F07FFEFAF0760
:101C0000FFEFBF0751F00197A109B109F1018687E4
:101C10009787A08BB18B81E08583A701960109C0CE
:101C200020E030E040E050E004C02FEF3FEF4FEF06
:101C30005FEFB901CA012496CDBFDEBFCF91DF911E
:101C40001F910F91FF90EF90DF90CF90BF90AF90DA
:101C50009F908F907F906F905F904F903F902F90CC
:101C60000895EF92FF920F931F93CF93DF93EC01B0
:101C70007A018B018EEF9FEFAFEFBFEFE80EF91EF9
:101C80000A1F1B1F8A8D9B8DAC8DBD8D0297A109EC
:101C9000B109E816F9060A071B0728F020E030E032
:101CA00040E050E012C02A8130E040E050E0C8013E
:101CB000B7010E9443469B01AC018EA19FA1A8A53C
:101CC000B9A5280F391F4A1F5B1FB901CA01DF914F
:101CD000CF911F910F91FF90EF900895AF92BF9217
:101CE000CF92DF92EF92FF920F931F93CF93DF93E8
:101CF0005C016B01DC0114966D937C93159716962D
:101D00004D915D916D917C9119974130510561051F
:101D1000710509F4D3C0ED91FC91828D938DA48D52
:101D2000B58D481759076A077B0708F0C7C04115EA
:101D300051056105710581F58081833049F442A127
:101D400053A164A175A1411551056105710521F5E6
:101D5000F50112861386148615860190F081E02D18
:101D600080859185C816D90608F0A8C0C60124E070
:101D7000969587952A95E1F7A0E0B0E022A133A1DE
:101D800044A155A1820F931FA41FB51FF50186879B
:101D90009787A08BB18B7AC08281082F10E094E0E6
:101DA000000F111F9A95E1F724C0CE010E94ED0AA1
:101DB000AB01BC014F3FFFEF5F07FFEF6F07FFEF86
:101DC0007F0711F481E07BC0423051056105710548
:101DD00008F474C0D501ED91FC91828D938DA48D92
:101DE000B58D481759076A077B0708F067C0C01A06
:101DF000D10AF501C081D181C016D106B0F6D50156
:101E00001A964D935D936D937C931D978EEFE82EFC
:101E10008FEFF82E8FEF082F8FEF182FE40EF51E9F
:101E2000061F171F8A8D9B8DAC8DBD8D0297A10952
:101E3000B109E816F9060A071B0728F020E030E090
:101E400040E050E012C02A8130E040E050E0C8019C
:101E5000B7010E9443469B01AC018EA19FA1A8A59A
:101E6000B9A5280F391F4A1F5B1FC60114E09695BC
:101E700087951A95E1F7A0E0B0E0280F391F4A1FB7
:101E80005B1FF50126873787408B518BFFE0CF2200
:101E9000DD24B5E0CC0CDD1CBA95E1F78EE290E0D4
:101EA000C80ED91ED5018D919C9111978C0D9D1D49
:101EB00052968D939C93539780E001C082E0DF910E
:101EC000CF911F910F91FF90EF90DF90CF90BF9037
:101ED000AF9008954F925F926F927F928F929F92F0
:101EE000AF92BF92CF92DF92EF92FF920F931F9328
:101EF000CF93DF93EC01D62E6C807D800894611C1B
:101F0000711C6114710409F44CC18E859F85A889E8
:101F1000B9890097A105B10509F443C11FE0412E1D
:101F2000512C462057204114510409F027C1019635
:101F3000A11DB11D8E879F87A88BB98B4A855B85B4
:101F40006C857D85E881F981411551056105710533
:101F500039F4808591856816790608F40FC121C18E
:101F6000828190E001979301A4E036952795AA9588
:101F7000E1F782239323892B09F000C1CF010E944E
:101F8000ED0A7B018C01623071058105910508F431
:101F90000AC18FEFE8168FEFF8068FEF08078FEF73
:101FA000180709F402C1E881F981828D938DA48D0F
:101FB000B58DE816F9060A071B0708F4A6C0DD2050
:101FC00009F4EFC04A855B856C857D85CF010E9451
:101FD0003E0D7B018C01611571058105910511F4A0
:101FE00087E0E4C091E0E916F1040105110509F468
:101FF000DAC0AFEFEA16AFEFFA06AFEF0A07AFEFBE
:102000001A0709F4D2C08881998140E050E060E06D
:1020100070E00E94E509882309F0C7C0E881F981D2
:10202000BE9680E092E001C011920197BFEF8F3F12
:102030009B07D1F7888099804EEFA42E4FEFB42EE6
:102040004FEFC42E4FEFD42EAE0CBF1CC01ED11EBE
:10205000F401828D938DA48DB58D0297A109B109EC
:10206000A816B906CA06DB0628F020E030E040E0FA
:1020700050E015C0D40112962C9130E040E050E0C1
:10208000C601B5010E9443469B01AC01F40186A143
:1020900097A1A0A5B1A5280F391F4A1F5B1FD40126
:1020A0009A962D933D934D935C939D97DD24CC247C
:1020B000C3941AC0C4828881998140E050E060E0F6
:1020C00070E00E94E509882309F06FC0E881F9817A
:1020D00082A593A5A4A5B5A50196A11DB11D82A7B2
:1020E00093A7A4A7B5A7D394E881F9818281D816D4
:1020F00008F382A593A5A4A5B5A58D199109A109F9
:10210000B10982A793A7A4A7B5A7EA86FB860C8787
:102110001D87C880D9808EEF9FEFAFEFBFEFE80E2D
:10212000F91E0A1F1B1FF601828D938DA48DB58D9C
:102130000297A109B109E816F9060A071B0728F05A
:1021400020E030E040E050E015C0D60112962C911E
:1021500030E040E050E0C801B7010E9443469B01D7
:10216000AC01F60186A197A1A0A5B1A5280F391F42
:102170004A1F5B1F2E873F87488B598B6C827D825D
:1021800035E0440C551C3A95E1F78EE290E0480E9C
:10219000591E88819981840D951D8A8B9B8B80E0C7
:1021A00005C084E003C082E001C081E0DF91CF91EF
:1021B0001F910F91FF90EF90DF90CF90BF90AF9065
:1021C0009F908F907F906F905F904F900895CF93E6
:1021D000DF93EC0194E01AC0888199810E94E5099F
:1021E000982F8823F1F4EA89FB898081882309F1FB
:1021F000853E29F08E3219F0838583FF16C0CE010B
:1022000060E00E946A0F982F882359F44E855F85FD
:10221000688979894115510561057105E9F69923A8
:1022200021F01E861F86188A198A892FDF91CF9187
:10223000089594E0F6CFCF93DF93EC0160E070E077
:102240000E946E0E482F8823E9F54E855F856889C8
:102250007989888199810E94E509482F882391F521
:10226000EA89FB89E081E53E89F1EE2379F1CE012F
:1022700061E00E946A0FE6CF6A897B89FB0180E2F8
:1022800090E001C0119201972FEF8F3F9207D1F795
:102290008C899D899C01D901FB012BE030E002C0B3
:1022A0008D918193215030408FEF2F3F3807C1F738
:1022B000EC89FD8983858871FB018487E881F98138
:1022C00081E08483842FDF91CF9108954E855F85CF
:1022D00068897989888199810E94E509482F882336
:1022E00059F2F0CFCF93DF93EC016C817D810E9496
:1022F0006E0E982F882399F44E855F8568897989B9
:10230000888199810E94E509982F882341F4EA8900
:10231000FB8985EE8083E881F98181E08483892FC0
:10232000DF91CF910895EF92FF920F931F93CF9378
:10233000DF93FC017B01EB01299686859785A089B7
:10234000B1890097A105B10509F471C0628973894B
:1023500080E090E0FB01E80FF91FE081E03241F0FE
:10236000E53009F4E5EEE99301968830910591F79F
:10237000DB0118968C91803211F48E0112C08EE22E
:10238000FE0181938F01FB019E012C5F3F4F8085F1
:10239000803239F0D8018D938D013196A217B307A1
:1023A000B1F7FB018385D70118968C93278D30E018
:1023B00040E050E0522F442733272227868D90E0BB
:1023C000A0E0B0E0DC0199278827282B392B4A2B85
:1023D0005B2B848D90E0A0E0B0E0282B392B4A2BBA
:1023E0005B2B958D80E0A0E0B0E0282B392B4A2BA9
:1023F0005B2BF7012083318342835383DB015996A2
:102400009C91599780E058962C91589730E0822BF8
:10241000932B8483958357969C91579780E056968B
:102420002C9130E0822B932B86839783E8011882CE
:10243000DF91CF911F910F91FF90EF9008955F92E0
:102440006F927F928F929F92AF92BF92CF92DF92C4
:10245000EF92FF920F931F93CF93DF93EC017B01D9
:1024600003C00894E11CF11CF70180818032C9F39C
:102470008F3211F08C3519F40894E11CF11C1E8286
:102480001F8218861986F7018081803240F4CE01C0
:1024900060E070E00E946E0E1A8A1B8A13C100E28F
:1024A00045E0542EAC89BD89FD018BE090E001C070
:1024B000019301972FEF8F3F9207D1F740E050E053
:1024C000CC24DD2438E0A32EB12C10E0F701EC0D74
:1024D000FD1D20810894C11CD11C213208F466C066
:1024E0002F3209F4FFC02C3509F4FCC02E3219F04C
:1024F0004A155B0584F088E0A816B10409F0DDC038
:102500002E3209F0DAC0110F110F48E050E02BE035
:10251000A22EB12CDBCF27FD1360822F81588F3183
:1025200018F08F558D3108F5F701EC0DFD1D308148
:10253000832F80548F3320F080548D3708F0BDC036
:10254000C5010197481759070CF0B7C00894C11C82
:10255000D11CFD01E40FF51F2083CA010196FD0186
:10256000E80FF91F3083AC011EC0622F70E0E0E07D
:10257000F0E201C031968081882329F090E086172F
:102580009707C1F79AC0822F81548A3110F41260E4
:1025900006C0822F81568A3110F411602052FD014D
:1025A000E40FF51F20834F5F5F4F90CF912F64E0C2
:1025B000452B09F482C08C91853E09F45C92E8E0D9
:1025C000AE16B10419F4912F990F990F292F30E00D
:1025D000C90183709070019709F460612C703070AC
:1025E0002430310509F468601B966C93CE0160E0DD
:1025F00070E00E946E0E482F882371F54E855F852E
:1026000068897989888199810E94E509482F882302
:1026100019F5EA89FB898081882311F444E01CC004
:10262000838583FD14C0DF018C899D899C01F9019C
:102630002BE030E0215030408FEF2F3F380761F022
:102640009C918081981719F411963196F3CFCE01A1
:1026500060E00E946A0FCFCFEC89FD89938594706A
:10266000442331F0842F443051F5992351F12AC08D
:10267000992329F5EA89FB89838584FF22C0EC0C24
:10268000FD1C75886624248930E02629372940E01E
:1026900050E0A90133272227938C8824828D90E073
:1026A00088299929A0E0B0E0282B392B4A2B5B2BF5
:1026B0002E833F8348875987F5CE86E003C0842F59
:1026C00001C085E0DF91CF911F910F91FF90EF90B6
:1026D000DF90CF90BF90AF909F908F907F906F9042
:1026E0005F900895912F60E063CF0F93CF93DF93B6
:1026F000EC019A01AB01BC01625D7F4F898101E071
:102700000E94AE06882311F063E06DC0C35DDD4F0B
:10271000988180E02A91CC52D24030E0822B932BDA
:1027200085559A4A11F062E05EC0C959DF4F288191
:1027300030E040E050E0522F4427332722278A918F
:1027400090E0A0E0B0E0DC0199278827282B392B06
:102750004A2B5B2B2297899190E0A0E0B0E0282BD8
:10276000392B4A2B5B2B9881C556D04080E0A0E0E6
:10277000B0E0282B392B4A2B5B2B50702654314468
:102780004445504011F460E02EC060E0CD57DF4F6B
:10279000288130E040E050E0522F442733272227A1
:1027A0008A9190E0A0E0B0E0DC0199278827282BEF
:1027B000392B4A2B5B2B2297899190E0A0E0B0E067
:1027C000282B392B4A2B5B2B988180E0A0E0B0E0CE
:1027D000282B392B4A2B5B2B50702654314444450F
:1027E000504009F061E0862FDF91CF910F9108955D
:1027F0006F927F928F929F92AF92BF92CF92DF9211
:10280000EF92FF920F931F93CF93DF93FC019B01F5
:10281000F42EA081B1818C91082F10E0005310405C
:102820000A30110568F411968C9111978A3341F49E
:102830001296A083B1830230110520F08BE091C283
:1028400000E010E0F801EE0FFF1FE653F84DC081E5
:10285000D181F901C083D183209711F48CE081C22A
:102860008881882379F08981882311F081E002C072
:102870008091572780FD06C0FF2009F46FC282FDBA
:102880006BC26CC21882F801EE0FFF1FE753FD4DBB
:10289000808189830E94C10580FF02C083E061C2FC
:1028A000FF2011F082FD58C2CE0140E050E060E010
:1028B00070E00E947513813021F0AA24BB246501C9
:1028C0003DC0000F111F07531D4DF8018181E82FF6
:1028D000F0E0A4E0EE0FFF1FAA95E1F7E451FE4FF0
:1028E000EC0FFD1F8481882309F43AC2838590E0B0
:1028F000A0E0B0E0D82ECC24BB24AA24828590E0AE
:10290000A0E0B0E0DC0199278827A82AB92ACA2AC2
:10291000DB2A808590E0A0E0B0E0A82AB92ACA2A84
:10292000DB2A918580E0A0E0B0E0A82AB92ACA2A73
:10293000DB2ACE01B601A5010E947513833011F484
:1029400081E00FC2882309F00BC29AAD80E029AD67
:1029500030E0822B932B8050924009F001C2CB5B78
:10296000DF4F988180E02A91C454D04030E0822B20
:10297000932B7C0100E010E0E114F1040105110546
:1029800041F5CB5ADF4F888190E0A0E0B0E0182FEE
:102990000027FF24EE248A9190E0A0E0B0E0DC0163
:1029A00099278827E82AF92A0A2B1B2B2297899135
:1029B00090E0A0E0B0E0E82AF92A0A2B1B2B9881CE
:1029C000C355D04080E0A0E0B0E0E82AF92A0A2B05
:1029D0001B2BEE8AFF8A088F198F2EAD2B8330E0D8
:1029E00040E050E0C801B7010E9443463B014C0162
:1029F0009DAD80E02CAD30E0822B932BA0E0B0E0C9
:102A00008A0D9B1DAC1DBD1D8E8F9F8FA8A3B9A3E2
:102A10008BAD8A83C05CDF4F9881C054D04080E08A
:102A20002FAD422F50E0482B592B48875987CE5B5A
:102A3000DF4F988180E02A91C154D04030E0822B52
:102A4000932B7C0100E010E0E114F1040105110575
:102A500041F5CF5ADF4F888190E0A0E0B0E0182F19
:102A60000027FF24EE248A9190E0A0E0B0E0DC0192
:102A700099278827E82AF92A0A2B1B2B2297899164
:102A800090E0A0E0B0E0E82AF92A0A2B1B2B9881FD
:102A9000CF54D04080E0A0E0B0E0E82AF92A0A2B29
:102AA0001B2B9DAD80E02CAD30E0822B932BA0E062
:102AB000B0E0E81AF90A0A0B1B0BE618F708080938
:102AC0001909F4E056954795FA95E1F7CA01A0E097
:102AD000B0E0E81AF90A0A0B1B0B2A8130E040E04B
:102AE00050E0C801B7010E9475462E5F3F4F4F4F1F
:102AF0005F4F2A8F3B8F4C8F5D8F273F8FE03807CA
:102B000080E0480780E0580710F411E007C0275F15
:102B10003F4F4040504008F033C112E08E8D9F8DF2
:102B2000A8A1B9A1860D971DA81DB91D8AA39BA3B5
:102B3000ACA3BDA388859985E4E096958795EA9531
:102B4000E1F7A0E0B0E02E8D3F8D48A159A1820FA2
:102B5000931FA41FB51F860D971DA81DB91D8EA319
:102B60009FA3A8A7B9A78FEF9FEFAFEFBFEF8E8707
:102B70009F87A88BB98B1C82133009F0DCC01D82A3
:102B8000C15ADF4F388120E08A91CE55D04090E085
:102B9000282B392B40E050E02A0D3B1D4C1D5D1DBC
:102BA0002A8B3B8B4C8B5D8BBE01625D7F4F898195
:102BB00001E00E94AE06882309F0BDC0C35DDD4F71
:102BC000988180E02A91CC52D24030E0822B932B26
:102BD00085559A4A09F0AFC029A930E040E050E09D
:102BE000522F44273327222788A990E0A0E0B0E0A5
:102BF000DC0199278827282B392B4A2B5B2B8EA5A4
:102C000090E0A0E0B0E0282B392B4A2B5B2B9FA54E
:102C100080E0A0E0B0E0282B392B4A2B5B2B22551B
:102C200032454146514409F086C0CB5EDD4F2881D4
:102C300030E040E050E0522F4427332722278A918A
:102C400090E0A0E0B0E0DC0199278827282B392B01
:102C50004A2B5B2B2297899190E0A0E0B0E0282BD3
:102C6000392B4A2B5B2B9881C351D24080E0A0E0E6
:102C7000B0E0282B392B4A2B5B2B2257324741449B
:102C8000514609F058C0C35EDD4F288130E040E076
:102C900050E0522F4427332722278A9190E0A0E06A
:102CA000B0E0DC0199278827282B392B4A2B5B2B96
:102CB0002297899190E0A0E0B0E0282B392B4A2B95
:102CC0005B2B9881CB51D24080E0A0E0B0E0282B74
:102CD000392B4A2B5B2B2A873B874C875D87C75E46
:102CE000DD4F288130E040E050E0522F4427332769
:102CF00022278A9190E0A0E0B0E0DC0199278827A4
:102D0000282B392B4A2B5B2B2297899190E0A0E04E
:102D1000B0E0282B392B4A2B5B2B9881C751D2402E
:102D200080E0A0E0B0E0282B392B4A2B5B2B2E87CC
:102D30003F87488B598B18831AA61BA61CA61DA675
:102D40008091CE279091CF2701968093CE279093A4
:102D5000CF278E839F8302C08AE003C080E001C03A
:102D60008DE0DF91CF911F910F91FF90EF90DF9059
:102D7000CF90BF90AF909F908F907F906F9008956D
:102D8000C35ADF4F288130E040E050E0522F442703
:102D9000332722278A9190E0A0E0B0E0DC01992758
:102DA0008827282B392B4A2B5B2B2297899190E07F
:102DB000A0E0B0E0282B392B4A2B5B2B9881CB5518
:102DC000D04080E0A0E0B0E0282B392B4A2B5B2BD1
:102DD0002AA33BA34CA35DA313E0ACCEFC01009758
:102DE000A9F08081882391F08681978186179707C3
:102DF00069F48181882311F081E002C08091572716
:102E000080FD02C080E0089583E0089589E0089580
:102E1000CF93DF93EB01823010F08BE017C0A82F27
:102E2000B0E0FD01EE0FFF1FE653F84D0190F08179
:102E3000E02D309709F01082209709F01882AA0F30
:102E4000BB1FA653B84DCD93DC9380E0DF91CF91AB
:102E500008955F926F927F928F929F92AF92BF92EE
:102E6000CF92DF92EF92FF920F931F93DF93CF9356
:102E7000CDB7DEB7A497CDBFDEBF3C016BA37CA36B
:102E8000DC011D921C925FE1552E54228E01035FDE
:102E90001F4F4E71CE018396B8010E94F81388230C
:102EA00011F0282F37C1CE01019689A39AA36BA1F7
:102EB0007CA1C8010E941F12282F452D50E0CA0195
:102EC0008C719070892B09F488C0222379F024300A
:102ED00009F020C1C8010E941B11282F882309F086
:102EE00019C1B8E05B2ACF8CD8A05BC052FE02C0EB
:102EF00028E010C1CF8CD8A0C114D10409F407C1B7
:102F0000F6018385817109F002C153FE4AC095899B
:102F100080E0248930E0822B932BA0E0B0E08C018C
:102F2000FF24EE24938D80E0228D30E0822B932BC2
:102F3000A0E0B0E0E82AF92A0A2B1B2B148A158A94
:102F4000128E138E148E158E168E178EED85FE85BD
:102F500081E0848382A493A4A4A4B5A4E114F10421
:102F600001051105A1F0CF01B801A7010E94C30C12
:102F7000282F882309F0CEC0ED85FE850894E1084E
:102F8000F10801091109E286F386048715878D850A
:102F90009E85B501A4010E94E509282F882309F028
:102FA000B9C053FE2CC0D6011B961C920E946D091D
:102FB000F6016687272F332727879C01442755274B
:102FC000208B692F772788279927618BED85FE85D0
:102FD00081E08483F0E25F2A12C0222309F09AC0C4
:102FE000CF8CD8A0C114D10409F493C0D6011B968C
:102FF0008C9184FD8EC051FE02C080FD88C0ED859D
:10300000FE8522A533A544A555A5D3015A962D9337
:103010003D934D935C935D978F8D98A15E968D93B4
:103020009C935F9714965C92D60155963C91559768
:1030300020E054968C91549790E0282B392B40E057
:1030400050E0A901332722275B969C915B9780E093
:103050005A966C9170E0862B972BA0E0B0E0282B5D
:10306000392B4A2B5B2BD3011E962D933D934D9309
:103070005C935197D6015F962C915F9730E040E0CA
:1030800050E0522F4427332722275E968C9190E000
:10309000A0E0B0E0DC0199278827282B392B4A2BA8
:1030A0005B2BD6015C968C9190E0A0E0B0E0282BE1
:1030B000392B4A2B5B2BD6015D969C9180E0A0E0DA
:1030C000B0E0282B392B4A2B5B2BD3011A962D937A
:1030D0003D934D935C931D9716961D921D921D92E4
:1030E0001C9219978FEF15968C93159756961D92F3
:1030F0001D921D921C925997ED93FC931197868116
:10310000978112968D939C93139720E003C027E03C
:1031100001C024E0822FA496CDBFDEBFCF91DF9106
:103120001F910F91FF90EF90DF90CF90BF90AF90E5
:103130009F908F907F906F905F9008952F923F9215
:103140004F925F926F927F928F929F92AF92BF92B7
:10315000CF92DF92EF92FF920F931F93DF93CF9363
:1031600000D00F92CDB7DEB78B839C83162F072F2D
:103170004A0129833A83D9011D921C92FC01628184
:103180007381808191810E94EE16782E882309F048
:10319000B4C1AB81BC8114968C9187FD66C080FD63
:1031A00003C007E0702EA9C1EB81FC812285338525
:1031B0004485558586819781A085B185281B390B6B
:1031C0004A0B5B0BC401A0E0B0E0281739074A079F
:1031D0005B0708F44901812F902F9C01290110E21F
:1031E000212E312C6B817C81260E371E82C1AB8152
:1031F000BC8116962D913D914D915C911997DA0104
:10320000C9019170A070B0700097A105B10509F0D7
:103210002CC1AB81BC81ED91FC91119715969C91CD
:10322000159782819817A0F12115310541055105A7
:1032300039F41E966D917D918D919C9151970BC0A3
:10324000AB81BC8152964D915D916D917C9155976A
:10325000CF010E94ED0A623071058105910540F4AD
:10326000EB81FC81848180688483B2E07B2E45C140
:103270006F3FFFEF7F07FFEF8F07FFEF9F0709F417
:10328000E0C0EB81FC81628B738B848B958B158204
:10329000AB81BC810D911C91119752962D913D915E
:1032A0004D915C9155972250304040405040F8017C
:1032B000828D938DA48DB58D0297A109B109281730
:1032C00039074A075B07B8F46280662D70E080E03A
:1032D00090E00E9443469B01AC01F80186A197A1B2
:1032E000A0A5B1A5280F391F4A1F5B1F2115310565
:1032F0004105510549F4AB81BC8114968C9114971A
:10330000806814968C93B1CFEB81FC818581590143
:103310006A01A80EB11CC11CD11C7401EF2CFF2442
:10332000E694E114F10409F453C0282F30E0C701FA
:10333000820F931F662D70E06817790718F47B01E0
:10334000E21AF30AD80111968C91B201A6019501F7
:103350000E2D0E94AE06EB81FC819481882319F02A
:103360009068948376C096FF29C0AB81BC81569645
:103370002D913D914D915C9159972A193B094C092A
:103380005D09C701A0E0B0E0281739074A075B07CD
:10339000A8F4F9E0220F331F441F551FFA95D1F707
:1033A000C201820F931FD101FC019C0120503E4FAE
:1033B00002C08D918193E217F307D9F7EB81FC816D
:1033C00085818E0D8583B701762F6627770F74C0B0
:1033D000AB81BC8114968C91149786FF1BC05696C6
:1033E0002D913D914D915C915997F8018181B101E9
:1033F00001E00E940E07AB81BC8114969C9114974A
:10340000882321F0906814969C9323C09F7BEB81C6
:10341000FC819483EB81FC8186899789A08DB18D95
:103420008A159B05AC05BD05B9F00190F081E02D32
:103430008181B101A601950101E00E94AE068823B9
:1034400059F0AB81BC8114968C91149780681496C6
:103450008C937724739451C0EB81FC81A68AB78A40
:10346000C08ED18E85818F5F8583AB81BC8116969E
:103470002D913D914D915C911997C9019170E0E0BA
:10348000F2E0E81BF90BB401E815F90508F4BF01F7
:103490008B01F901F170B0968B819C81E80FF91FC7
:1034A000920104C08191D9018D939D01015010407A
:1034B000BFEF0F3F1B07B1F7460E571ECB01A0E031
:1034C000B0E0EB81FC812681378140855185280F52
:1034D000391F4A1F5B1F2683378340875187E98145
:1034E000FA8180819181860F971F80839183861A4C
:1034F000970A8114910409F07ACE872D2496CDBFC6
:10350000DEBFCF91DF911F910F91FF90EF90DF9081
:10351000CF90BF90AF909F908F907F906F905F9073
:103520004F903F902F9008952F923F924F925F922D
:103530006F927F928F929F92AF92BF92CF92DF92C3
:10354000EF92FF920F931F93DF93CF9300D00F92D0
:10355000CDB7DEB78B839C83162F072F4A012983B3
:103560003A83D9011D921C92FC0162817381808192
:1035700091810E94EE16682E882309F002C2AB8169
:10358000BC8114968C9187FD7CC081FD03C057E0FF
:10359000652EF7C1EB81FC812285338544855585F5
:1035A000C401A0E0B0E0820F931FA41FB51F8217D3
:1035B0009307A407B50710F488249924812F902F2E
:1035C0009C01290140E2242E312C6B817C81260E46
:1035D000371EB2C1AB81BC8116962D913D914D91A4
:1035E0005C911997DA01C9019170A070B0700097D1
:1035F000A105B10509F058C1AB81BC81ED91FC91E9
:10360000119715969C9115978281981708F454C0CC
:103610002115310541055105C9F41E966D917D9125
:103620008D919C9151976115710581059105F9F472
:10363000CF0140E050E060E070E00E943E0DEB8181
:10364000FC8166877787808B918B0BC0AB81BC81B7
:1036500052964D915D916D917C915597CF010E944D
:103660003E0D611571058105910509F469C161304F
:1036700071058105910541F4EB81FC8184818068AD
:10368000848332E0632E7DC16F3FFFEF7F07FFEF42
:103690008F07FFEF9F0749F4AB81BC8114968C9193
:1036A0001497806814968C93EEC0EB81FC81628B3A
:1036B000738B848B958B1582AB81BC8114968C9116
:1036C000149786FF1BC0ED91FC91119756962D9192
:1036D0003D914D915C9159978181B10101E00E942A
:1036E0000E07EB81FC819481882319F09068948304
:1036F000CAC09F7BAB81BC8114969C93EB81FC81FB
:1037000000811181228933894489558922503040B2
:1037100040405040F801828D938DA48DB58D029765
:10372000A109B109281739074A075B07B8F4728065
:10373000672D70E080E090E00E9443469B01AC0161
:10374000F80186A197A1A0A5B1A5280F391F4A1F8E
:103750005B1F211531054105510549F4AB81BC8141
:1037600014968C911497806814968C938ACFEB8171
:10377000FC81858169017A01C80ED11CE11CF11C14
:103780005401AB2CBB24A694A114B10409F453C07A
:10379000282F30E0C501820F931F672D70E0681756
:1037A000790718F45B01A21AB30AD80111968C911B
:1037B000B201A70196010A2D0E940E07882309F085
:1037C0005DC0AB81BC8156962D913D914D915C9130
:1037D00059972C193D094E095F09C501A0E0B0E0D9
:1037E000281739074A075B07C8F499E0220F331FEF
:1037F000441F551F9A95D1F7F201E20FF31FD10133
:103800009F0120503E4F02C081918D93E217F30734
:10381000D9F7EB81FC8184818F7B8483AB81BC8170
:1038200015968C9115978A0D15968C93B501762F68
:103830006627770F64C0EB81FC8186899789A08D0C
:10384000B18D8C159D05AE05BF0501F1268137812F
:103850004085518582859385A485B58528173907CC
:103860004A075B0798F4D80111968C91B101A70122
:10387000960101E00E94AE06882341F0EB81FC81B5
:10388000848180688483662463947BC0AB81BC811F
:103890005696CD92DD92ED92FC92599715968C91A9
:1038A00015978F5F15968C93EB81FC81268137816C
:1038B00040855185C901917060E072E0681B790B09
:1038C000CB01B4018815990508F4BC018B01F901FD
:1038D000F170B0968B819C81E80FF91F920104C0B2
:1038E000D9018D919D01819301501040BFEF0F3F91
:1038F0001B07B1F7EB81FC81848180648483460ED1
:10390000571ECB01A0E0B0E0EB81FC81268137811E
:1039100040855185280F391F4A1F5B1F2683378337
:1039200040875187E981FA8180819181860F971FB5
:1039300080839183861A970A8114910409F04ACEF4
:10394000AB81BC8116962D913D914D915C9119975B
:103950001A968D919D910D90BC91A02D8217930781
:10396000A407B50730F4EB81FC81228733874487B5
:103970005587AB81BC8114968C9114978062149604
:103980008C93862D2496CDBFDEBFCF91DF911F9102
:103990000F91FF90EF90DF90CF90BF90AF909F90EE
:1039A0008F907F906F905F904F903F902F900895F1
:1039B0000F931F93CF93DF93EC016A817B81888102
:1039C00099810E94EE16982F882309F072C08C818D
:1039D00085FF6FC086FF14C0E881F981BE01605E7B
:1039E0007F4F2E893F89488D598D818101E00E944A
:1039F0000E07882311F091E05CC08C818F7B8C8353
:103A00004A8D5B8D6C8D7D8D888199810E94E50941
:103A1000982F882309F04DC00E8D1F8DF8018385E6
:103A2000806283878A85848F8B85858F8A859B8535
:103A3000AC85BD85CD01AA27BB27868F8A859B854E
:103A4000AC85BD858B2F9927AA27BB27878F8E85AD
:103A5000828F8F85838F8E859F85A889B989CD01B7
:103A6000AA27BB27848B8E859F85A889B989CD011C
:103A7000AA27BB27892F9927858B0E946D09F801FA
:103A8000668B272F3327278B9C0144275527208FB0
:103A9000692F772788279927618F8C818F7D8C8369
:103AA000E881F98181E08483888199810E945E0A9E
:103AB000982F892FDF91CF911F910F910895CF9368
:103AC000DF93EC010E94D81C882311F4188219821C
:103AD000DF91CF9108952F923F924F925F926F9214
:103AE0007F928F929F92AF92BF92CF92DF920F936D
:103AF0001F93DF93CF93CDB7DEB72897CDBFDEBF3F
:103B00008F8398873A014B01DC0112966D917C916D
:103B100013978D919C910E94EE16182F882309F01F
:103B2000F3C1EF81F885848187FD98C0AF81B885A6
:103B30001A96AD90BD90CD90DC901D97A614B70459
:103B4000C804D90410F481FF02C064015301EF815D
:103B5000F885268137814085518516821782108627
:103B600011868FEF8583A114B104C104D10409F437
:103B70005FC10190F081E02DE983FA838281682E94
:103B800077248824992489E0660C771C881C991C6A
:103B90008A95D1F72115310541055105F1F119013A
:103BA0002A0108942108310841085108C601B501CD
:103BB0006150704080409040A40193010E9475467E
:103BC0002B833C834D835E83C201B101A401930129
:103BD0000E9475468B819C81AD81BE8182179307BF
:103BE000A407B507D0F088279927DC018619970923
:103BF000A809B90982219321A421B521EF81F88573
:103C000086839783A087B187A81AB90ACA0ADB0AF4
:103C1000428953896489758939C0AF81B8851E96F8
:103C20004D915D916D917C915197411551056105C3
:103C3000710521F589819A8140E050E060E070E0F3
:103C40000E943E0DAB01BC0141305105610571057B
:103C500039F4EF81F88584818068848312E054C14F
:103C60004F3FFFEF5F07FFEF6F07FFEF7F07B1F1F8
:103C7000EF81F88546875787608B718BAF81B88558
:103C800052964D935D936D937C93559741155105D5
:103C90006105710509F058C0CBC0EF81F8858481BA
:103CA0002081318181FF0DC0C9010E943E0DAB0111
:103CB000BC01411551056105710541F464015301D1
:103CC00049C0C9010E94ED0AAB01BC014F3FFFEFA3
:103CD0005F07FFEF6F07FFEF7F0749F4AF81B885FC
:103CE00014968C911497806814968C93EDC0423092
:103CF00051056105710508F4ACCFAF81B885ED9130
:103D0000FC91828D938DA48DB58D481759076A0754
:103D10007B0708F09ECFAF81B88552964D935D9397
:103D20006D937C935597FD0186819781A085B18520
:103D3000860D971DA81DB91D86839783A087B1871F
:103D4000A618B708C808D9086A147B048C049D0417
:103D500008F4A3CFEF81F88586819781A085B1858E
:103D60008A0D9B1DAC1DBD1D86839783A087B187DF
:103D7000D601C50109E0B695A795979587950A954F
:103D8000D1F7082F85838FEF91E0A0E0B0E0A82263
:103D9000B922CA22DB22A114B104C104D10409F45E
:103DA00047C080809180EEEFAE2EEFEFBE2EEFEF9A
:103DB000CE2EEFEFDE2EA40EB51EC61ED71EF401CA
:103DC000828D938DA48DB58D0297A109B109A81696
:103DD000B906CA06DB06C0F4228130E040E050E0BC
:103DE000C601B5010E9443469B01AC01F40186A1C6
:103DF00097A1A0A5B1A5280F391F4A1F5B1F211548
:103E000031054105510549F4AF81B88514968C916F
:103E10001497806814968C9321CF59016A01A00EE3
:103E2000B11CC11CD11C0F5FEF81F885058303C055
:103E3000AA24BB246501EF81F88586819781A0853E
:103E4000B1859170A070B0700097A105B10509F41B
:103E500045C026893789408D518DA216B306C40608
:103E6000D506E1F1848186FF1AC00190F081E02D32
:103E70006F817885605E7F4F818101E00E940E072F
